:020000040000FA
:0408000025EF06F0EA
:1008100003B207EF05F0F2B422EF05F09EB02AEF25
:1008200005F09EB232EF05F0F2A81AEF04F0F2B232
:100830001CEF04F003EF06F0CD90F2929EA026EF9D
:1008400004F00101463F26EF04F0472B85C189F1F2
:1008500086C18AF187C18BF188C18CF181C185F194
:1008600082C186F183C187F184C188F17DC181F1A4
:100870007EC182F17FC183F180C184F179C17DF1B4
:100880007AC17EF17BC17FF17CC180F175C179F1C4
:1008900076C17AF177C17BF178C17CF171C175F1D4
:1008A00072C176F173C177F174C178F16DC171F1E4
:1008B0006EC172F16FC173F170C174F1CECF6DF181
:1008C000CFCF6EF146C16FF147C170F1CF6ACE6AEA
:1008D0000101466B476B9E90CD800EBC0E8E0EBA0A
:1008E00075EF04F00E8A03EF06F00E8C0EBEB1EF2A
:1008F00004F06DC171F16EC172F16FC173F170C11D
:1009000074F171C175F172C176F173C177F174C17F
:1009100078F175C179F176C17AF177C17BF178C14F
:100920007CF179C17DF17AC17EF17BC17FF17CC11F
:1009300080F17DC181F17EC182F17FC183F180C1EF
:1009400084F181C185F182C186F183C187F184C1BF
:1009500088F185C189F186C18AF187C18BF188C18F
:100960008CF10101516B526B536B546B6D515127DC
:100970006E5152236F51532370515423715151279B
:10098000725152237351532374515423755151277B
:10099000765152237751532378515423795151275B
:1009A0007A5152237B5153237C5154237D5151273B
:1009B0007E5152237F51532380515423815151271B
:1009C00082515223835153238451542385515127FB
:1009D00086515223875153238851542389515127DB
:1009E0008A5152238B5153238C515423D890543322
:1009F000533352335133D8905433533352335133EA
:100A0000D890543353335233513303EF06F00392EB
:100A1000030103EE00F080517F0BE92604C0EFFFD5
:100A2000802B8151805D700BD8A48B820000805197
:100A3000815D700BD8A48B9281518019D8B4079036
:100A400003EF06F0F2940101383F03EF06F0392B73
:100A500003EF06F09E900101463F03EF06F0472B9F
:100A600003EF06F09E92C3CF48F1C4CF49F1C28292
:100A700007B465EF05F03AC13EF13BC13FF13CC11F
:100A800040F13DC141F151C155F152C156F153C13F
:100A900057F154C158F16DC159F16EC15AF16FC18E
:100AA0005BF170C15CF1010148514E2749514F2360
:100AB000E86A50230D2E65EF05F04FC14AF150C191
:100AC0004BF14E6B4F6B506B078E0201002F03EF03
:100AD00006F03C0E006F0101616776EF05F062677A
:100AE00076EF05F0636776EF05F064677AEF05F05F
:100AF000AAEF05F065C100F166C101F167C102F11D
:100B000068C103F10101010E046F000E056F000EB4
:100B1000066F000E076F04EC13F000C165F101C110
:100B200066F102C167F103C168F100679FEF05F04C
:100B300001679FEF05F002679FEF05F00367AAEFDB
:100B400005F061C165F162C166F163C167F164C11D
:100B500068F10E80D57ED5BE54D0D6CF3AF1D7CF2E
:100B60003BF138C13CF1E86AE8CF3DF10F8001016B
:100B700047A7C7EF05F00E9A0E9C0E9E0101000ECE
:100B8000516F600E526F3D0E536F080E546F01018E
:100B90003ABFD7EF05F03B67D7EF05F03C67D7EFDB
:100BA00005F03D67D7EF05F0F288FCEF05F0F2980D
:100BB000516B526B536B546B6D6B6E6B6F6B706BD9
:100BC000716B726B736B746B756B766B776B786B29
:100BD000796B7A6B7B6B7C6B7D6B7E6B7F6B806BD9
:100BE000816B826B836B846B856B866B876B886B89
:100BF000896B8A6B8B6B8C6BD76AD66A0101386BF9
:100C0000396B03EF06F002C0E0FF005001C0D8FFCF
:100C10001000A6B209EF06F00CC0A9FF0BC0A8FF98
:100C2000A69EA69CA684F29E550EA76EAA0EA76E3F
:100C3000A682F28EA694A6B21BEF06F01200A96E51
:100C4000A69EA69CA680A8501200076A0E6A0F6A8C
:100C50000F010E0EC16E860EC06E030EC26E0F0126
:100C6000896A110E926E080E8A6EF10E936E8B6A6F
:100C7000800E946EF18E0D6A01014E6B4F6B506BBE
:100C80004A6B4B6B0F01280ED56EF28AB00ECD6EFB
:100C90009D800101516B526B536B546B556B566BBE
:100CA000576B586B5D6B5E6B5F6B606B0E9A0E9C47
:100CB0000E9E760ECA6E9D8202013C0E006FCC6ABB
:100CC000160E1FEC06F0E8CF00F1170E1FEC06F031
:100CD000E8CF01F1180E1FEC06F0E8CF02F1190E73
:100CE0001FEC06F0E8CF03F1010103AF92EF06F02D
:100CF000FBEC13F0160E0C6E00C10BF009EC06F0C5
:100D0000170E0C6E01C10BF009EC06F0180E0C6EFC
:100D100002C10BF009EC06F0190E0C6E03C10BF0CA
:100D200009EC06F000C161F101C162F102C163F199
:100D300003C164F100C165F101C166F102C167F14F
:100D400003C168F11A0E1FEC06F0E8CF00F11B0E8C
:100D50001FEC06F0E8CF01F11C0E1FEC06F0E8CF07
:100D600002F11D0E1FEC06F0E8CF03F1010103AF05
:100D7000E8EF06F0FBEC13F01A0E0C6E00C10BF05E
:100D800009EC06F01B0E0C6E01C10BF009EC06F02D
:100D90001C0E0C6E02C10BF009EC06F01D0E0C6E61
:100DA00003C10BF009EC06F01A0E1FEC06F0E8CFB9
:100DB00000F11B0E1FEC06F0E8CF01F11C0E1FEC3A
:100DC00006F0E8CF02F11D0E1FEC06F0E8CF03F1AC
:100DD00000C169F101C16AF102C16BF103C16CF19B
:100DE000240EAC6E900EAB6E240EAC6E080EB86E78
:100DF000000EB06E1F0EAF6E0401806B816B0F0191
:100E0000900EAB6E0F019D8A0301806B816BA26B0C
:100E10008B9207900001F28EF28C07B0C8EF10F0B1
:100E20000EB0E8EF0BF00301805181197F0BD8B4AD
:100E3000C8EF10F013EE00F081517F0BE126812BFB
:100E4000E7CFE8FFE00BD8B4C8EF10F023EE82F054
:100E5000A2511F0BD926E7CFDFFFA22BDF50780A64
:100E6000D8A4C8EF10F0078065C100F166C101F198
:100E700067C102F168C103F10101040E046F000EA5
:100E8000056F000E066F000E076F04EC13F000AF45
:100E900053EF07F00101030E656F000E666F000E41
:100EA000676F000E686F03018251720AD8B4E8EFD1
:100EB0000BF08251520AD8B4E8EF0BF08251750A58
:100EC000D8B4E8EF0BF08251630AD8B484EF0DF088
:100ED0008251690AD8B4EDEF08F082517A0AD8B489
:100EE00000EF0AF08251490AD8B48CEF08F0825121
:100EF000500AD8B4AAEF07F08251700AD8B4EDEFC7
:100F000007F08251540AD8B418EF08F08251740ADD
:100F1000D8B45EEF08F08251730AD8B418EF0BF022
:100F20008251530AD8B47DEF0BF0B9EF0DF00401F4
:100F300014EE00F080517F0BE12682C4E7FF802B86
:100F400012000D0E826F97EC07F00A0E826F97EC7D
:100F500007F0120083C31EF184C31FF185C320F183
:100F600086C321F187C322F188C323F189C324F109
:100F70008AC325F18BC326F18CC327F1010149EC0B
:100F800014F0C0EC13F0160E0C6E00C10BF009EC5F
:100F900006F0170E0C6E01C10BF009EC06F0180EEE
:100FA0000C6E02C10BF009EC06F0190E0C6E03C1B9
:100FB0000BF009EC06F000C161F101C162F102C160
:100FC00063F103C164F100C165F101C166F102C1C1
:100FD00067F103C168F18CEF08F083C31EF184C38D
:100FE0001FF185C320F186C321F187C322F188C395
:100FF00023F189C324F18AC325F18BC326F18CC365
:1010000027F1010149EC14F0C0EC13F000C161F1CB
:1010100001C162F102C163F103C164F100C165F174
:1010200001C166F102C167F103C168F18CEF08F0FC
:1010300083C31EF184C31FF185C320F186C321F150
:1010400087C322F188C323F189C324F18AC325F120
:101050008CC326F18DC327F1010149EC14F0C0ECDB
:1010600013F00101000E046F000E056F010E066FF4
:10107000000E076F13EC13F01A0E0C6E00C10BF08C
:1010800009EC06F01B0E0C6E01C10BF009EC06F02A
:101090001C0E0C6E02C10BF009EC06F01D0E0C6E5E
:1010A00003C10BF009EC06F000C169F101C16AF15E
:1010B00002C16BF103C16CF18CEF08F083C31EF128
:1010C00084C31FF185C320F186C321F187C322F1B8
:1010D00088C323F189C324F18AC325F18CC326F187
:1010E0008DC327F1010149EC14F0C0EC13F00101AC
:1010F000000E046F000E056F010E066F000E076FE5
:1011000013EC13F000C169F101C16AF102C16BF186
:1011100003C16CF18CEF08F0160E1FEC06F0E8CF5F
:1011200000F1170E1FEC06F0E8CF01F1180E1FECCE
:1011300006F0E8CF02F1190E1FEC06F0E8CF03F13C
:101140009EEC13F0CAEC11F00401730E826F97EC61
:1011500007F004012C0E826F97EC07F061C100F1DB
:1011600062C101F163C102F164C103F19EEC13F0AD
:10117000CAEC11F00401730E826F97EC07F00401C2
:101180002C0E826F97EC07F01A0E1FEC06F0E8CFDA
:1011900000F11B0E1FEC06F0E8CF01F11C0E1FEC56
:1011A00006F0E8CF02F11D0E1FEC06F0E8CF03F1C8
:1011B000D4EC0DF004012C0E826F97EC07F069C19E
:1011C00000F16AC101F16BC102F16CC103F1D4EC11
:1011D0000DF0A1EC07F0B9EF0DF00401690E826F7C
:1011E00097EC07F004012C0E826F97EC07F00101D9
:1011F000040E006F000E016F000E026F000E036FF1
:101200009EEC13F020C182F40401300E822797EC8B
:1012100007F021C182F40401300E822797EC07F019
:1012200022C182F40401300E822797EC07F023C11B
:1012300082F40401300E822797EC07F024C182F477
:101240000401300E822797EC07F025C182F40401D7
:10125000300E822797EC07F026C182F40401300E8D
:10126000822797EC07F027C182F40401300E822711
:1012700097EC07F004012C0E826F97EC07F0010148
:10128000030E006F000E016F000E026F000E036F61
:101290009EEC13F020C182F40401300E822797ECFB
:1012A00007F021C182F40401300E822797EC07F089
:1012B00022C182F40401300E822797EC07F023C18B
:1012C00082F40401300E822797EC07F024C182F4E7
:1012D0000401300E822797EC07F025C182F4040147
:1012E000300E822797EC07F026C182F40401300EFD
:1012F000822797EC07F027C182F40401300E822781
:1013000097EC07F004012C0E826F97EC07F00101B7
:10131000150E006F000E016F000E026F000E036FBE
:101320009EEC13F020C182F40401300E822797EC6A
:1013300007F021C182F40401300E822797EC07F0F8
:1013400022C182F40401300E822797EC07F023C1FA
:1013500082F40401300E822797EC07F024C182F456
:101360000401300E822797EC07F025C182F40401B6
:10137000300E822797EC07F026C182F40401300E6C
:10138000822797EC07F027C182F40401300E8227F0
:1013900097EC07F004012C0E826F97EC07F0200EFB
:1013A000F86EF76AF66A04010900F5CF82F497EC4B
:1013B00007F00900F5CF82F497EC07F00900F5CFAC
:1013C00082F497EC07F00900F5CF82F497EC07F070
:1013D0000900F5CF82F497EC07F00900F5CF82F40D
:1013E00097EC07F00900F5CF82F497EC07F00900BD
:1013F000F5CF82F497EC07F0A1EC07F0B9EF0DF010
:101400008351630AD8A4B9EF0DF08451610AD8A4BE
:10141000B9EF0DF085516C0AD8A4B9EF0DF08651E3
:10142000410A42E08651440A1BE08651420AD8B480
:1014300067EF0AF08651350AD8B443EF0FF08651B2
:10144000360AD8B498EF0FF08651370AD8B401EFB6
:1014500010F08651380AD8B45FEF10F0B9EF0DF0F4
:101460000798079A04017A0E826F97EC07F004013F
:10147000780E826F97EC07F00401640E826F97EC90
:1014800007F081A84BEF0AF00401550E826F97EC2C
:1014900007F050EF0AF004014C0E826F97EC07F052
:1014A000A1EC07F0B9EF0DF00788079A04017A0E56
:1014B000826F97EC07F00401410E826F97EC07F002
:1014C0000401610E826F97EC07F041EF0AF0079874
:1014D000078A04017A0E826F97EC07F00401420E2E
:1014E000826F97EC07F00401610E826F97EC07F0B2
:1014F00041EF0AF00101620E046F010E056F000E4C
:10150000066F000E076F5DC100F15EC101F15FC1A2
:1015100002F160C103F104EC13F003BFD7EF0AF04E
:101520000E0E1FEC06F0E8CF0CF10F0E1FEC06F0CC
:10153000E8CF0DF1100E1FEC06F0E8CF0EF1110E02
:101540001FEC06F0E8CF0FF14DEC12F05DC104F195
:101550005EC105F15FC106F160C107F104EC13F053
:10156000078211EC12F04DEC12F0079211EC12F020
:101570005DC100F15EC101F15FC102F160C103F123
:10158000079211EC12F0CC0E046FE00E056F870E7F
:10159000066F050E076F04EC13F000C10CF101C1DA
:1015A0000DF102C10EF103C10FF10FEF0BF00101BC
:1015B000800E006F1A0E016F060E026F000E036F91
:1015C00042C104F143C105F144C106F145C107F12F
:1015D00004EC13F003AFF0EF0AF0FBEC13F0120091
:1015E0000E0E1FEC06F0E8CF0CF10F0E1FEC06F00C
:1015F000E8CF0DF1100E1FEC06F0E8CF0EF1110E42
:101600001FEC06F0E8CF0FF142C100F143C101F138
:1016100044C102F145C103F1078211EC12F00CC183
:1016200000F10DC101F10EC102F10FC103F1120071
:101630000401730E826F97EC07F004012C0E826F89
:1016400097EC07F0078455C15DF156C15EF157C1B3
:101650005FF158C160F13EC142F13FC143F140C169
:1016600044F141C145F14AC14CF14BC14DF10794E0
:101670003EEC0BF0A1EC07F0B9EF0DF05DC100F10D
:101680005EC101F15FC102F160C103F101019EEC95
:1016900013F0CAEC11F00401630E826F97EC07F0AF
:1016A00004012C0E826F97EC07F042C100F143C198
:1016B00001F144C102F145C103F101019EEC13F0B7
:1016C000CAEC11F00401660E826F97EC07F004017A
:1016D0002C0E826F97EC07F0FBEC13F04CC100F17D
:1016E0004DC101F101019EEC13F0CAEC11F00401AF
:1016F000740E826F97EC07F012000F820401530EF4
:10170000826F97EC07F004012C0E826F97EC07F0C4
:1017100083C31EF184C31FF185C320F186C321F169
:1017200087C322F188C323F189C324F18AC325F139
:101730008BC326F18CC327F1010149EC14F0C0ECF6
:1017400013F000C15DF101C15EF102C15FF103C19F
:1017500060F18EC31EF18FC31FF190C320F191C3BE
:1017600021F192C322F193C323F194C324F195C3D1
:1017700025F196C326F197C327F1010149EC14F036
:10178000C0EC13F000C142F101C143F102C144F1C8
:1017900003C145F13CEC14F099C323F19AC324F141
:1017A0009BC325F19CC326F19DC327F1010149ECA0
:1017B00014F0C0EC13F000C14CF101C14DF13EEC4E
:1017C0000BF004012C0E826F97EC07F0EFEF0BF09B
:1017D0008251520A03E10E82EFEF0BF00E9282511A
:1017E000750A03E10F84F6EF0BF00F9407840FB234
:1017F0001BEF0CF00FA407EF0CF059C15DF15AC1BB
:101800005EF15BC15FF15CC160F10FEF0CF055C19F
:101810005DF156C15EF157C15FF158C160F13EC143
:1018200042F13FC143F140C144F141C145F14AC1D8
:101830004CF14BC14DF107940EA03DEF0CF00101AE
:1018400069672AEF0CF06A672AEF0CF06B672AEFE2
:101850000CF06C672EEF0CF03DEF0CF07AEC0AF018
:1018600069C104F16AC105F16BC106F16CC107F1F0
:1018700004EC13F003BF81EF0DF07AEC0AF00101E4
:10188000000E046F000E056F010E066F000E076F4D
:1018900032EC13F00FA454EF0CF00401750E826FBC
:1018A00097EC07F059EF0CF00401720E826F97EC81
:1018B00007F004012C0E826F97EC07F09EEC13F0FA
:1018C0001D6768EF0CF00401200E826F6BEF0CF0C7
:1018D00004012D0E826F97EC07F024C182F40401FD
:1018E000300E822797EC07F025C182F40401300EF8
:1018F000822797EC07F004012E0E826F97EC07F019
:1019000026C182F40401300E822797EC07F027C12C
:1019100082F40401300E822797EC07F004016D0E6B
:10192000826F97EC07F004012C0E826F97EC07F0A2
:1019300042C100F143C101F144C102F145C103F1CB
:1019400001019EEC13F0CAEC11F00401480E826F05
:1019500097EC07F004017A0E826F97EC07F0040110
:101960002C0E826F97EC07F05DC100F15EC101F1B2
:101970005FC102F160C103F101019EEC13F0CAECFA
:1019800011F00401630E826F97EC07F004012C0E36
:10199000826F97EC07F05DC100F15EC101F15FC19C
:1019A00002F160C103F101010A0E046F000E056F20
:1019B000000E066F000E076F13EC13F0000E046F9D
:1019C000120E056F000E066F000E076F32EC13F05B
:1019D0009EEC13F01EC182F40401300E822797ECB6
:1019E00007F01FC182F40401300E822797EC07F044
:1019F00020C182F40401300E822797EC07F021C148
:101A000082F40401300E822797EC07F022C182F4A1
:101A10000401300E822797EC07F023C182F4040101
:101A2000300E822797EC07F024C182F40401300EB7
:101A3000822797EC07F004012E0E826F97EC07F0D7
:101A400025C182F40401300E822797EC07F026C1ED
:101A500082F40401300E822797EC07F027C182F44C
:101A60000401300E822797EC07F00401730E826F99
:101A700097EC07F004012C0E826F97EC07F0FBEC5B
:101A800013F04CC100F14DC101F1E3EC0EF00EB2C8
:101A90004DEF0DF00EA07FEF0DF004012C0E826FC4
:101AA00097EC07F0200EF86EF76AF66A0401090059
:101AB000F5CF82F497EC07F00900F5CF82F497ECAC
:101AC00007F00900F5CF82F497EC07F00900F5CF95
:101AD00082F497EC07F00900F5CF82F497EC07F059
:101AE0000900F5CF82F497EC07F00900F5CF82F4F6
:101AF00097EC07F00900F5CF82F497EC07F0A1EC22
:101B000007F00E90B9EF0DF00401630E826F97ECB1
:101B100007F004012C0E826F97EC07F0BFEC0DF07C
:101B200004012C0E826F97EC07F032EC0EF00401EA
:101B30002C0E826F97EC07F0AEEC0EF004012C0E29
:101B4000826F97EC07F00101F80E006FCD0E016F68
:101B5000660E026F030E036FD4EC0DF004012C0E21
:101B6000826F97EC07F0C4EC0EF0A1EC07F0B9EF30
:101B70000DF00301A26B07900F92C8EF10F0D89000
:101B80000E0E1FEC06F0E8CF00F10F0E1FEC06F072
:101B9000E8CF01F1100E1FEC06F0E8CF02F1110EB4
:101BA0001FEC06F0E8CF03F10101000E046F000EF8
:101BB000056F010E066F000E076F32EC13F09EECFE
:101BC00013F01EC182F40401300E822797EC07F057
:101BD0001FC182F40401300E822797EC07F020C168
:101BE00082F40401300E822797EC07F021C182F4C1
:101BF0000401300E822797EC07F022C182F4040121
:101C0000300E822797EC07F023C182F40401300ED6
:101C1000822797EC07F024C182F40401300E82275A
:101C200097EC07F025C182F40401300E822797EC6F
:101C300007F004012E0E826F97EC07F026C182F4A4
:101C40000401300E822797EC07F027C182F40401CB
:101C5000300E822797EC07F004016D0E826F97EC2F
:101C600007F01200120E1FEC06F0E8CF00F1130E81
:101C70001FEC06F0E8CF01F1140E1FEC06F0E8CFE0
:101C800002F1150E1FEC06F0E8CF03F101010A0E78
:101C9000046F000E056F000E066F000E076F13EC49
:101CA00013F0000E046F120E056F000E066F000E8B
:101CB000076F32EC13F09EEC13F01EC182F40401A6
:101CC000300E822797EC07F01FC182F40401300E1A
:101CD000822797EC07F020C182F40401300E82279E
:101CE00097EC07F021C182F40401300E822797ECB3
:101CF00007F022C182F40401300E822797EC07F02E
:101D000023C182F40401300E822797EC07F024C12E
:101D100082F40401300E822797EC07F004012E0EA6
:101D2000826F97EC07F025C182F40401300E822700
:101D300097EC07F026C182F40401300E822797EC5D
:101D400007F027C182F40401300E822797EC07F0D8
:101D50000401730E826F97EC07F012000A0E1FEC5D
:101D600006F0E8CF00F10B0E1FEC06F0E8CF01F112
:101D70000C0E1FEC06F0E8CF02F10D0E1FEC06F082
:101D8000E8CF03F1E3EF0EF0060E1FEC06F0E8CF0C
:101D900000F1070E1FEC06F0E8CF01F1080E1FEC72
:101DA00006F0E8CF02F1090E1FEC06F0E8CF03F1D0
:101DB000E3EF0EF00101FBEC13F007844AC100F1E0
:101DC0004BC101F107940101E80E046F800E056F0D
:101DD000000E066F000E076F13EC13F0000E046F79
:101DE000040E056F000E066F000E076F32EC13F045
:101DF000880E046F130E056F000E066F000E076F3E
:101E000004EC13F00A0E046F000E056F000E066F4F
:101E1000000E076F32EC13F09EEC13F001011D670A
:101E200017EF0FF00401200E826F1AEF0FF004017C
:101E30002D0E826F97EC07F024C182F40401300E5E
:101E4000822797EC07F025C182F40401300E822727
:101E500097EC07F026C182F40401300E822797EC3C
:101E600007F004012E0E826F97EC07F027C182F471
:101E70000401300E822797EC07F00401430E826FB5
:101E800097EC07F0120087C31EF188C31FF189C3C6
:101E900020F18AC321F18BC322F18CC323F18DC3BE
:101EA00024F18EC325F190C326F191C327F10101DE
:101EB0001D6B49EC14F0C0EC13F00101000E046F2F
:101EC000000E056F010E066F000E076F13EC13F086
:101ED0000E0E0C6E00C10BF009EC06F00F0E0C6E2E
:101EE00001C10BF009EC06F0100E0C6E02C10BF0F4
:101EF00009EC06F0110E0C6E03C10BF009EC06F0B4
:101F000004017A0E826F97EC07F004012C0E826FA9
:101F100097EC07F00401350E826F97EC07F004018F
:101F20002C0E826F97EC07F0BFEC0DF050EF0AF02B
:101F300087C31EF188C31FF189C320F18AC321F131
:101F40008BC322F18CC323F18DC324F18EC325F101
:101F500090C326F191C327F101011D6B49EC14F0E8
:101F6000C0EC13F0880E046F130E056F000E066FA1
:101F7000000E076F08EC13F0000E046F040E056FDF
:101F8000000E066F000E076F13EC13F00101E80E50
:101F9000046F800E056F000E066F000E076F32ECA7
:101FA00013F00A0E0C6E00C10BF009EC06F00B0EDC
:101FB0000C6E01C10BF009EC06F00C0E0C6E02C1A8
:101FC0000BF009EC06F00D0E0C6E03C10BF009ECE2
:101FD00006F004017A0E826F97EC07F004012C0ED4
:101FE000826F97EC07F00401360E826F97EC07F0D2
:101FF00004012C0E826F97EC07F0AEEC0EF050EF60
:102000000AF087C31EF188C31FF189C320F18AC378
:1020100021F18BC322F18CC323F18DC324F18FC333
:1020200025F190C326F191C327F1010149EC14F089
:10203000C0EC13F0000E046F120E056F000E066F59
:10204000000E076F13EC13F001010A0E046F000E6F
:10205000056F000E066F000E076F32EC13F0120EC4
:102060000C6E00C10BF009EC06F0130E0C6E01C1F2
:102070000BF009EC06F0140E0C6E02C10BF009EC2B
:1020800006F0150E0C6E03C10BF009EC06F004010E
:102090007A0E826F97EC07F004012C0E826F97EC9A
:1020A00007F00401370E826F97EC07F004012C0E45
:1020B000826F97EC07F032EC0EF050EF0AF087C316
:1020C0001EF188C31FF189C320F18AC321F18BC39C
:1020D00022F18CC323F18DC324F18EC325F190C36B
:1020E00026F191C327F101011D6B49EC14F0C0ECFE
:1020F00013F0880E046F130E056F000E066F000EAE
:10210000076F08EC13F0000E046F040E056F000E4D
:10211000066F000E076F13EC13F00101E80E046F59
:10212000800E056F000E066F000E076F32EC13F085
:10213000060E0C6E00C10BF009EC06F0070E0C6EDB
:1021400001C10BF009EC06F0080E0C6E02C10BF099
:1021500009EC06F0090E0C6E03C10BF009EC06F059
:1021600004017A0E826F97EC07F004012C0E826F47
:1021700097EC07F00401380E826F97EC07F004012A
:102180002C0E826F97EC07F0C4EC0EF050EF0AF0C3
:1021900081A886EF11F007A83FEF11F00101800E32
:1021A000006F1A0E016F060E026F000E036F3EC124
:1021B00004F13FC105F140C106F141C107F104EC52
:1021C00013F003BF86EF11F0C4EC11F03EC100F133
:1021D0003FC101F140C102F141C103F1078211EC9D
:1021E00012F00CC104F10DC105F10EC106F10FC1D1
:1021F00007F1F80E006FCD0E016F660E026F030E31
:10220000036F04EC13F00E0E0C6E00C10BF009EC22
:1022100006F00F0E0C6E01C10BF009EC06F0100E6B
:102220000C6E02C10BF009EC06F0110E0C6E03C12E
:102230000BF009EC06F007840101FBEC13F04AC136
:1022400000F14BC101F107940A0E0C6E00C10BF0B6
:1022500009EC06F00B0E0C6E01C10BF009EC06F058
:102260000C0E0C6E02C10BF009EC06F00D0E0C6E9C
:1022700003C10BF009EC06F0079886EF11F007AAEE
:1022800086EF11F007840101FBEC13F04AC100F165
:102290004BC101F10794060E0C6E00C10BF009EC66
:1022A00006F0070E0C6E01C10BF009EC06F0080EEB
:1022B0000C6E02C10BF009EC06F0090E0C6E03C1A6
:1022C0000BF009EC06F0078455C100F156C101F18D
:1022D00057C102F158C103F10794120E0C6E00C1F0
:1022E0000BF009EC06F0130E0C6E01C10BF009ECBB
:1022F00006F0140E0C6E02C10BF009EC06F0150E80
:102300000C6E03C10BF009EC06F0079A0401805132
:1023100081197F0B0BE09EA809D014EE00F08151CB
:102320007F0BE126E750812B0F01AD6E0DEF07F01B
:102330000CC100F10DC101F10EC102F10FC103F199
:10234000000E046F000E056F010E066F000E076F82
:1023500032EC13F01DA1C3EF11F01451D8B4C3EF48
:1023600011F00CC100F10DC101F10EC102F10FC15C
:1023700003F1000E046F000E056F0A0E066F000ECB
:10238000076F32EC13F0120001010C6B0D6B0E6B3A
:102390000F6B12001EC182F40401300E822797ECED
:1023A00007F01FC182F40401300E822797EC07F07A
:1023B00020C182F40401300E822797EC07F021C17E
:1023C00082F40401300E822797EC07F022C182F4D8
:1023D0000401300E822797EC07F023C182F4040138
:1023E000300E822797EC07F024C182F40401300EEE
:1023F000822797EC07F025C182F40401300E822772
:1024000097EC07F026C182F40401300E822797EC86
:1024100007F027C182F40401300E822797EC07F001
:1024200012000101005305E1015303E1025301E1F0
:10243000002BD4EC12F0FBEC13F02C51006F2D515B
:10244000016F420E046F4B0E056F000E066F000EFB
:10245000076F13EC13F000C104F101C105F102C1D3
:1024600006F103C107F10CC100F10DC101F10EC16C
:1024700002F10FC103F107B242EF12F008EC13F0C2
:1024800044EF12F004EC13F000C10CF101C10DF1A6
:1024900002C10EF103C10FF11200FBEC13F04CC1AD
:1024A00000F14DC101F1060E1FEC06F0E8CF04F17A
:1024B000070E1FEC06F0E8CF05F1080E1FEC06F042
:1024C000E8CF06F1090E1FEC06F0E8CF07F104ECA7
:1024D00013F000C118F101C119F102C11AF103C1D1
:1024E0001BF1290E046F000E056F000E066F000E23
:1024F000076F13EC13F0EE0E046F430E056F000E22
:10250000066F000E076F08EC13F018C104F119C133
:1025100005F11AC106F11BC107F113EC13F000C15C
:1025200010F101C111F102C112F103C113F1120E38
:102530001FEC06F0E8CF04F1130E1FEC06F0E8CF15
:1025400005F1140E1FEC06F0E8CF06F1150E1FEC96
:1025500006F0E8CF07F10D0E006F000E016F000EC0
:10256000026F000E036F13EC13F0180E046F000ED1
:10257000056F000E066F000E076F32EC13F010C1EE
:1025800004F111C105F112C106F113C107F108EC04
:1025900013F06A0E046F2A0E056F000E066F000E10
:1025A000076F04EC13F01200BF0EFA6E200E2D6FB1
:1025B0002C6BD8900037013702370337D8B0E5EFDE
:1025C00012F02D2FDAEF12F02C072D070353D8B499
:1025D00012000331070B8009326F03390F0B010F13
:1025E0002C6F80EC5FF0336F2C0580EC5FF0335D77
:1025F000335F2C6B3233D8B02C272C3332A9FAEF4F
:1026000012F033512C27120020EC14F0D8B0120035
:1026100003510719286FE3EC13F0D8900751031901
:1026200028AF800F1200286B07EC14F0D8A01DEC27
:1026300014F0D8B01200F2EC13F0FBEC13F01F0E04
:10264000296F33EC14F00B35D8B0E3EC13F0D8A0BD
:102650000335D8B01200292F21EF13F028B10AEC6E
:1026600014F01200286B045105110611071100081F
:10267000D8A007EC14F0D8A01DEC14F0D8B01200CC
:10268000086B096B0A6B0B6B33EC14F01F0E296F90
:1026900033EC14F007510B5DD8A45BEF13F0065137
:1026A0000A5DD8A45BEF13F00551095DD8A45BEF78
:1026B00013F00451085DD8A06EEF13F00451085FC9
:1026C0000551D8A0053D095F0651D8A0063D0A5F17
:1026D0000751D8A0073D0B5FD8900081292F48EF04
:1026E00013F028B10AEC14F0286B07EC14F0D89022
:1026F00037EC14F007510B5DD8A48BEF13F00651A3
:102700000A5DD8A48BEF13F00551095DD8A48BEFB7
:1027100013F00451085DD8A09AEF13F0003F9AEF30
:1027200013F0013F9AEF13F0023F9AEF13F0032BDF
:10273000D8B4120028B10AEC14F012000101286B81
:1027400007EC14F0D8B012003CEC14F0200E296F06
:10275000003701370237033711EE27F00A0E2A6FD0
:10276000E7360A0EE75CD8B0E76EE5522A2FB0EFE5
:1027700013F0292FA8EF13F028B11D81D890120073
:1027800001010A0E286F200E296F11EE1DF028514D
:102790002A6F0A0ED890E652D8B0E726E7322A2FE1
:1027A000CBEF13F00333023301330033292FC5EF8E
:1027B00013F0E750FF0FD8A00335D8B012001DB1B9
:1027C0000AEC14F01200045100270551D8B0053D61
:1027D00001270651D8B0063D02270751D8B0073D62
:1027E000032712000051086F0151096F02510A6F4F
:1027F00003510B6F12000101006B016B026B036B45
:1028000012000101046B056B066B076B12000335A8
:10281000D8A012000351800B001F011F021F031FCD
:10282000003F1AEF14F0013F1AEF14F0023F1AEFC5
:1028300014F0032B282B032512000735D8A0120013
:102840000751800B041F051F061F071F043F30EFB1
:1028500014F0053F30EF14F0063F30EF14F0072B73
:10286000282B0725120000370137023703370837B6
:1028700009370A370B37120001011D6B1E6B1F6BE6
:10288000206B216B226B236B246B256B266B276BD4
:1028900012001E510F0B1E6F1F510F0B1F6F205187
:1028A0000F0B206F21510F0B216F22510F0B226F45
:1028B00023510F0B236F24510F0B246F25510F0B46
:1028C000256F26510F0B266F27510F0B276F120014
:10BF0000E844F926000C160C2B0C3F0C520C640C68
:10BF1000760C860C960CA50CB30CC10CCF0CDC0C6B
:06BF2000E80CF40C000C1B
:00000001FF
